:100000000C94C8010C9400020C9400020C940002A1
:100010000C9400020C9400020C9400020C94000258
:100020000C9400020C9400020C9476220C94482349
:100030000C9400020C9400020C9400020C94000238
:100040000C9400020C9400020C9400020C94000228
:100050000C9400020C94FB1D0C9400020C94000202
:100060000C9400020C9400020C9400020C94000208
:100070000C9400020C9400020C9400020C940002F8
:100080000C94FF050C9400020C9400020C940002E6
:100090000C9400020C9400020C9400020C940002D8
:1000A0000C9400020C9400020C940002B406960614
:1000B00099069C069F06A206A506A806AB06AE06F4
:1000C000B106E107E707ED07F207F707FC070108AC
:1000D00006080B08100815081A081F0825081B0D2C
:1000E0001B0D470D470DAF0DDA0EDA0EDA0ECD0DF2
:1000F000660E770E770EB523DC23D424DC23D424BC
:1001000028244B24D424A224B12400030501020492
:10011000A0FF60FF4DFFB3FF33FFCDFF00000010D5
:1001200010101000201020001E001F0020002100D1
:10013000220023000000000000000000000000007A
:1001400000000000000000000000000000000000AF
:100150000000000000000000000101010101010198
:10016000010102020202020202020203030303036C
:10017000030303040404040404040505050505063B
:1001800006060606070707070708080808090909F9
:10019000090A0A0A0B0B0B0C0C0C0D0D0D0E0E0EA2
:1001A0000F0F0F1010111111121213131414151533
:1001B00016161717181819191A1A1B1B1C1D1D1EA5
:1001C0001E1F2020212222232424252626272829F9
:1001D000292A2B2C2D2D2E2F303132323334353627
:1001E0003738393A3B3C3D3E3F4041424344454627
:1001F0004748494A4C4D4E4F505153545556585903
:100200005A5B5D5E5F616264656668696B6C6D6FA9
:100210007072737577787A7B7D7E8082838587881C
:100220008A8C8E8F91939596989A9C9EA0A2A3A556
:10023000A7A9ABADAFB1B3B5B7BABCBEC0C2C4C657
:10024000C9CBCDCFD1D4D6D8DBDDDFE2E4E7E9EB13
:10025000EEF0F3F5F8FAFDFF2003520041004D00E7
:100260004100200057004F0052004B005300200077
:100270004D0036002D0042000000160352004100E0
:100280004D004100200057004F0052004B0053002A
:1002900000000403090409023B00020100A0FA095E
:1002A00004000001030101000921110100012240A5
:1002B0000007058103080001090401000103000093
:1002C00000092111010001226D00070582032000B1
:1002D00001120100020000000841526B0001000100
:1002E00002000105010980A101850319012AB70057
:1002F000150126B700950175108100C0050C090194
:10030000A101850419012AA002150126A002950168
:1003100075108100C005010906A1018506050719B0
:10032000E029E715002501950875018102050719E7
:100330000029EF1500250195F075018102050819C6
:10034000012905950575019102950175039101C07B
:1003500005010906A101050719E029E71500250196
:10036000950875018102950175088101050719003D
:1003700029FF150026FF009506750881000508195C
:10038000012905950575019102950175039101C03B
:1003900011241FBECFEFDAE0DEBFCDBF04B603FEEF
:1003A00018C08091C2029091C302A091C402B09182
:1003B000C5028730904BA740B04B59F41092C2024F
:1003C0001092C3021092C4021092C502E0E0F8E35A
:1003D000099511E0A0E0B1E0ECEAFCE402C0059070
:1003E0000D92AA3AB107D9F722E0AAEAB1E001C01A
:1003F0001D92A23CB207E1F70E942C1A0C945426DD
:100400000C9400000E94C4020C9447190F931F9390
:10041000CF93DF93EC018B010E94C307C0318FE5BE
:10042000D80729F0C131EFE5DE0749F01EC0F80119
:100430008281882311F081E007C081E013C0F801B8
:100440008281882371F082E00E941E1043E062E006
:1004500081E00E94C50A80E0DF91CF911F910F914A
:10046000089582E00E943F10F1CFB801CE01DF91E4
:10047000CF911F910F910C94230ACF93C82F0E9404
:10048000FD028C2FCF910C94430B81E00C94FA0267
:1004900080E00C94FA0283E290E00E94D12582323F
:1004A00081F484E290E00E94D125823051F485E20B
:1004B00090E00E94D12591E0873109F090E0892FEA
:1004C00001C080E0817008950E944B02882319F0DA
:1004D0000E94C90602C00E94D1060E94D9060E944D
:1004E000E1020C94F402CF93C82F811102C06FEF88
:1004F00001C062E283E290E00E94EF25C11102C0D8
:100500006FEF01C062E084E290E00E94EF25C1112C
:1005100002C06FEF01C067E185E290E0CF910C94DB
:10052000EF250E94640281E00E9473020C94491935
:10053000E82FF0E0EE0FFF1FE45EFE4F8491DB0139
:100540008C933196E4911196EC930895E82FF0E0A6
:10055000EE0FFF1FE05FFE4F8491DB018C9331961D
:10056000E4911196EC930895882321F08FEFDA013E
:100570008C9308956630D0F7E62FF0E0E65FFE4FEB
:10058000E491DA01EC9308950C943409CF93DF934E
:100590001F92CDB7DEB7AE014F5F5F4F0E94B4022E
:1005A000E981F0E0EF57FD4F10821092AE011092FA
:1005B000AF011092B0011092B1010F90DF91CF9175
:1005C00008958091AD0181110EC081E08093AD014D
:1005D0008DE0809391009FB7F89423E020939900D9
:1005E000809398009FBF0895E1E7F0E080818260EA
:1005F000808308958093B70108958093B60108958C
:100600008091B2019091B301A091B401B091B50174
:1006100080739927AA27BB2724E0B695A7959795BD
:1006200087952A95D1F782309105A105B10571F022
:1006300083309105A105B10569F040E00197A1055E
:10064000B10511F060E008C06FEF02C04FEF60E04D
:1006500080E003C04FEF6FEF8FEF0C941A0940E07A
:1006600060E080E00C941A09E5E0F1E065817681B4
:1006700082810E94C108482F872F0C941A09DF92AB
:10068000EF92FF920F931F93CF93DF9300D0CDB7DC
:10069000DEB780910C0190E020910A01821B910944
:1006A0008038910514F09A9505C081382FEF920794
:1006B0000CF4939597FD0396959587959595879559
:1006C000182F80910D0190E020910B01821B910960
:1006D00097FD03969595879595958795082FD090CA
:1006E0000701E12CF12CBE016F5F7F4F8E2D0E9420
:1006F00098028A8182958F7060910A01819F600DB6
:10070000112470910B01809F700D11248D2D0E947A
:10071000C108462F282F672FC7010E940B098FEFB2
:10072000E81AF80A26E0E216F104E9F60F900F90B5
:10073000DF91CF911F910F91FF90EF90DF9008957F
:10074000AF92BF92CF92DF92EF92FF920F931F93DF
:10075000CF93DF93082F10910A0180910C0190E054
:10076000811B910997FD039695958795959587959A
:10077000D82FB0900B0180910D0190E08B19910959
:1007800097FD03969595879595958795C82F0E9417
:10079000A42566E070E00E941C25E12CF12C6C0180
:1007A000DD24011103C0EC14FD04C9F40E94A4254A
:1007B0008370A12E8D9FA00C11240E94A42583700C
:1007C0007B2D8C9F700D11246A2D809107010E9452
:1007D000C108462F282F672FC7010E940B098FEFF2
:1007E000E81AF80A86E0E816F104D9F6DF91CF910D
:1007F0001F910F91FF90EF90DF90CF90BF90AF903F
:100800000895DF92EF92FF920F931F93CF93DF93A0
:100810008091B2019091B301A091B401B091B50162
:100820000090090104C0880F991FAA1FBB1F0A94DA
:10083000D2F7D82EC1E8D2E000E010E08FE3E82E36
:10084000F12C899124E0829FC0011124803491050C
:1008500024F4B701681B790B02C060E070E06D0DF5
:100860007FEF809107010E94C108462F282F672F34
:10087000C8010E940B090F5F1F4F0630110509F7D1
:10088000DF91CF911F910F91FF90EF90DF9008952E
:100890008F929F92AF92BF92CF92DF92EF92FF9290
:1008A0000F931F93CF93DF9300D0CDB7DEB7809126
:1008B000B2019091B301A091B401B091B501009043
:1008C000090104C0880F991FAA1FBB1F0A94D2F701
:1008D000B82EA090070181E8E82E82E0F82E00E013
:1008E00010E09FE3C92ED12CF70181917F01F4E044
:1008F0008F9FC00111248034910524F44601881A89
:10090000990A02C0812C912CBE016F5F7F4F802F0E
:100910000E94980269816B0D680D7FEF8A2D0E94FD
:10092000C108462F282F672FC8010E940B090F5FAF
:100930001F4F06301105C1F60F900F90DF91CF9138
:100940001F910F91FF90EF90DF90CF90BF90AF90ED
:100950009F908F9008958F929F92AF92BF92CF9267
:10096000DF92EF92FF920F931F93CF93DF9300D00C
:10097000CDB7DEB78091B2019091B301A091B401DF
:10098000B091B5010090090104C0880F991FAA1FFA
:10099000BB1F0A94D2F7B82EA090070181E8E82E79
:1009A00082E0F82E00E010E09FE3C92ED12CF70181
:1009B00081917F01F4E08F9FC00111248034910563
:1009C00024F44601881A990A02C0812C912CBE0198
:1009D0006F5F7F4F802F0E9498026A816B0D680DB8
:1009E0007FEF8A2D0E94C108462F282F672FC8014C
:1009F0000E940B090F5F1F4F06301105C1F60F90C3
:100A00000F90DF91CF911F910F91FF90EF90DF90AA
:100A1000CF90BF90AF909F908F900895EF92FF92EC
:100A20000F931F93CF93DF93F82E0E94A42566E0C7
:100A300070E00E941C25C0E0D0E08C011127F1106D
:100A400003C00C171D0789F40E94A425E82E0E94FC
:100A5000A4256E2D782F809107010E94C108462F92
:100A6000282F672FCE010E940B092196C630D10591
:100A700031F7DF91CF911F910F91FF90EF90089583
:100A8000EF92FF920F931F93CF93DF9300D0CDB7D8
:100A9000DEB78091B2019091B301A091B401B09101
:100AA000B5010090090104C0880F991FAA1FBB1F40
:100AB0000A94D2F7F82EE090070100E010E0BE01A2
:100AC0006F5F7F4F802F0E94A60269816F0D7A8130
:100AD0008E2D0E94C108462F282F672FC8010E9423
:100AE0000B090F5F1F4F0630110549F70F900F904C
:100AF000DF91CF911F910F91FF90EF900895EF92AA
:100B0000FF920F931F93CF93DF9300D0CDB7DEB743
:100B10008091B2019091B301A091B401B091B5015F
:100B20000090090104C0880F991FAA1FBB1F0A94D7
:100B3000D2F7F82EE090070100E010E0BE016F5FF1
:100B40007F4F802F0E94A60269816F0D67FD60951F
:100B50006695669580910A01680F7A81769571583D
:100B60008E2D0E94C108462F282F672FC8010E9492
:100B70000B090F5F1F4F0630110501F70F900F9003
:100B8000DF91CF911F910F91FF90EF900895CF9239
:100B9000DF92EF92FF920F931F93CF93DF931F92F9
:100BA000CDB7DEB785E0E82E81E0F82E10E0F70142
:100BB000678D70A1809107010E94C108D62E072F72
:100BC000C82EAE014F5F5F4F612F80E00E94B402DC
:100BD00089812C2D4D2D602F90E00E940B091F5F05
:100BE000F2E0EF0EF11C163011F70F90DF91CF916C
:100BF0001F910F91FF90EF90DF90CF9008951F927B
:100C00000F920FB60F9211240F931F932F933F93C0
:100C10004F935F936F937F938F939F93AF93BF9304
:100C2000EF93FF938091AC01843120F48F5F809328
:100C3000AC019CC08091B2019091B301A091B4012C
:100C4000B091B5010196A11DB11D8093B2019093A1
:100C5000B301A093B401B093B5018091AE0190911E
:100C6000AF01A091B001B091B1018F3F2FEF92077A
:100C7000A207B20759F00196A11DB11D8093AE01E4
:100C80009093AF01A093B001B093B101E1E8F2E01D
:100C900080818F3F11F08F5F8083319682E0E7384B
:100CA000F807B1F7E0910801EF3F19F40E94000343
:100CB0005DC08091B701882321F08091050185FDF9
:100CC0001EC0809106018823E1F020EB34E0829F72
:100CD000A001839F500D1124052E000C660B770B8D
:100CE00081E00091AE011091AF012091B0013091EF
:100CF000B101401751076207730720F002C081E07D
:100D000001C080E080FDE0E081E0909104019E134D
:100D100001C080E0E09304014E2F50E04B305105BC
:100D200018F5FA01EA5AFF4F0C9452250E94340339
:100D30001DC00E94C7051AC00E943F0317C00E9431
:100D4000A00314C00E94010411C00E9448040EC0F8
:100D50000E94AB040BC00E940E0508C00E94400513
:100D600005C00E947F0502C00E942F03FF91EF91F2
:100D7000BF91AF919F918F917F916F915F914F91B3
:100D80003F912F911F910F910F900FBE0F901F90C9
:100D900018954BE250E067E270E085E091E00C943A
:100DA000C1254BE250E067E270E085E091E00C94F1
:100DB000DF250E9443090E94E908E1E8F2E08FEF95
:100DC0008083818382838383848385830895809154
:100DD000080190E001968B30910514F08AE090E0D4
:100DE000809308010C94D1068091080190E001974E
:100DF00097FF02C080E090E08B30910514F08AE00C
:100E000090E0809308010C94D1068091090190E054
:100E100001968430910514F083E090E080930901FD
:100E20000C94D1068091090190E0019797FF02C0D0
:100E300080E090E08430910514F083E090E08093AE
:100E400009010C94D1068091070190E008968F3F2C
:100E5000910519F014F08FEF90E0809307010C9446
:100E6000D1068091070190E0089797FF02C080E0CB
:100E700090E08F3F910519F014F08FEF90E0809390
:100E800007010C94D10680910A0190E008968F3FEB
:100E9000910519F014F08FEF90E080930A010C9403
:100EA000D10680910A0190E0089797FF02C080E088
:100EB00090E08F3F910519F014F08FEF90E0809350
:100EC0000A010C94D10680910B0190E008968F3FA7
:100ED000910519F014F08FEF90E080930B010C94C2
:100EE000D10680910B0190E0089797FF02C080E047
:100EF00090E08F3F910519F014F08FEF90E0809310
:100F00000B010C94D10680910C0190E008968F3F64
:100F1000910519F014F08FEF90E080930C010C9480
:100F2000D10680910C0190E0089797FF02C080E005
:100F300090E08F3F910519F014F08FEF90E08093CF
:100F40000C010C94D10680910D0190E008968F3F22
:100F5000910519F014F08FEF90E080930D010C943F
:100F6000D10680910D0190E0089797FF02C080E0C4
:100F700090E08F3F910519F014F08FEF90E080938F
:100F80000D010C94D1060F931F93CF93DF93EC01C7
:100F90008B01DB0112968C911297882329F06C91BA
:100FA00011968C910E94C602FE01FF55EE30F105AC
:100FB00008F050C0EF59FF4FD8011296CC910C9415
:100FC0005225CC2309F447C00E9423073CC0CC2300
:100FD00009F441C00E94310736C0CC23E1F10E94E0
:100FE000E70631C0CC23B9F10E94F4062CC0CC2313
:100FF00091F10E94050727C0CC2369F10E941207D6
:1010000022C0CC2341F10E9443071DC0CC2319F11B
:101010000E94510718C0CC23F1F00E94630713C04F
:10102000CC23C9F00E94710716C0CC23A1F00E9406
:10103000830709C0CC2379F00E94910704C0CC2318
:1010400051F00E94A307C0E006C0CC2321F00E940B
:10105000B10701C0C1E08C2FDF91CF911F910F919B
:101060000895EF92FF920F931F93CF93DF938B011D
:10107000682F11110AC0442329F0E82FF0E0E85A44
:10108000FE4F6491762F862F75C0212F30E0E82F18
:10109000F0E0442321F0E85AFE4FE491F0E046E00E
:1010A000049FC0011124CFEFD0E0BE010E940825AB
:1010B0004BEA4603C001479F900D1124800F911DFC
:1010C000800F911D982F990F890FAE01421B530B72
:1010D0004E9FD0014F9FB00D5E9FB00D11249B2FEE
:1010E000189FA0011124452F55278E01041B150BB5
:1010F0000E9FA0010F9F500D1E9F500D11247E01C9
:10110000E81AF108E29E8001E39E100DF29E100D98
:101110001124212F3327C21BD30BCE9F9001CF9FC9
:10112000300DDE9F300D112462307105A9F048F4B6
:101130006115710569F061307105C9F48B2F752F48
:101140000DC06430710581F058F06630710579F496
:101150007E2F8B2F932F0DC0832F7B2F9E2F09C0A7
:101160008E2F7B2F952F05C08E2F732F02C07E2FC1
:10117000852F692FDF91CF911F910F91FF90EF90F5
:10118000089541E00E9431080895E9E9F2E0808382
:10119000618324E630E042E050E0BF0188EA0C942D
:1011A000FA0921E020939902EAE9F2E09C012E5E1F
:1011B0003F4FDC014D91CD014193A217B307C9F711
:1011C00024E630E043E150E069E972E088EA0C94FB
:1011D000FA09CF9360E087E10E94C50861E080E0F2
:1011E0000E94C508C0E0CF5F60E08C2F0E94C50858
:1011F000C231C9F76FE383E10E94C5086FE384E160
:101200000E94C5086FE385E10E94C50861E086E1A0
:10121000CF910C94C508FC01EE0FFF1F8E0F9F1F8E
:10122000FC01E957FD4F60834183228381E0809375
:10123000B8010895FF920F931F93CF93DF93182F58
:10124000062FF42EC0E0D0E02F2D402F612FCE01CD
:101250000E940B092196C630D105B1F7DF91CF91DD
:101260001F910F91FF9008958091B801882341F05C
:1012700087E892E00E94D10861E086E10E94C508FB
:101280001092B80108951092B9008CE08093B800D4
:1012900008959F92AF92BF92CF92DF92EF92FF920A
:1012A0000F931F93CF93DF93B82EEB010E94D41DB1
:1012B0006C01C431D10558F0CF3F8FEFD80759F0FA
:1012C000CE0164E170E00E9408257B0107C0EE2496
:1012D000E394F12C03C025E0E22EF12C84E8A82E43
:1012E00094EA992E1092BC009092BC000E94D41DEA
:1012F0008C018091BC0087FD08C00E94D41D801B1A
:10130000910B8E159F05A8F32AC08091B900887FA4
:10131000883041F08091B900887F803119F00FEF5B
:101320001FEF1FC0B092BB00A092BC000E94D41D52
:101330008C018091BC0087FD08C00E94D41D801BD9
:10134000910B8E159F05A8F30AC08091B900887F84
:10135000883111F0803419F700E010E00EC00EEF74
:101360001FEFCF3F8FEFD80709F4BCCFC6010E9413
:10137000EC1D8C179D0708F4B5CFC801DF91CF9104
:101380001F910F91FF90EF90DF90CF90BF90AF90A3
:101390009F9008950F931F93CF93DF93EB0180935A
:1013A000BB0084E88093BC000E94D41D8C01809116
:1013B000BC0087FD0EC0CF3F8FEFD807C1F30E945E
:1013C000D41D801B910B8C179D0788F38EEF9FEF28
:1013D0000CC02091B900287F81E090E0283211F400
:1013E00080E090E0919581959109DF91CF911F91D7
:1013F0000F910895CF92DF92EF92FF920F931F9378
:10140000CF93DF936B018A017901B9010E944909E9
:10141000E6010C0D1D1DC017D10761F424E92093CE
:10142000BC00DF91CF911F910F91FF90EF90DF9063
:10143000CF90089597FDF2CFB70189910E94CA0914
:10144000EACF81E0089581E0089508950C94250A7B
:101450001F93CF93DF9300D000D01F92CDB7DEB79C
:1014600049835A836B833091BA0189819A81311102
:1014700014C0662359F0222349F00E941511182F39
:10148000682F89819A810E94BC1003C00E94E810D5
:10149000182F69817A81812F04C00E9415116981FA
:1014A0007A810F900F900F900F900F90DF91CF9156
:1014B0001F910C940A18FC01262F408151816281F2
:1014C000738184810C94280A81E00895CF93DF937F
:1014D000EC0160E00E945B0ABE01DF91CF910C94A9
:1014E000260A8F929F92AF92BF92CF92DF92EF9295
:1014F000FF920F931F936B017C0181E090E0A0E0CD
:10150000B0E04C015D0104C0880C991CAA1CBB1CF6
:101510004A95D2F7AC01BD0104C0440F551F661FA8
:10152000771F2A95D2F7482959296A297B2904C0AF
:10153000880F991FAA1FBB1F0A95D2F78A019B012A
:101540000C211D212E213F214017510762077307EF
:1015500039F4BC01CD016C297D298E299F290AC04F
:1015600080959095A095B095BC01CD016C217D2111
:101570008E219F211F910F91FF90EF90DF90CF90D0
:10158000BF90AF909F908F9008950F93382F262F84
:101590006091C0017091C1018091C2019091C3011D
:1015A000042F432F0E94710A0F910C94F80F0C9492
:1015B00091020C94020208950E94660F0E94DB0AB9
:1015C0002FEF84E39CE0215080409040E1F700C081
:1015D00000000C94211E0F931F93CF93DF938C0177
:1015E00061E00E945B0AEC01B8010E9406028823B8
:1015F000F1F1B801CE010E94251C8823C1F1B80188
:10160000CE010E94391A882391F1B801CE010E94BF
:10161000811B882361F1F8018281882309F1CB3590
:101620008DE5D807C1F050F4C115FCE5DF0781F066
:10163000CF3DDC45A9F40E944C1619C0CC35EDE530
:10164000DE0761F0CD35DD4559F40E948F1508C0E5
:101650000E94DC0A0CC00E94981502C00E949B15D3
:10166000C801DF91CF911F910F910C94210A80E066
:10167000DF91CF911F910F9108950C9445020E9424
:10168000520B0C944802089581E008950C94440B89
:101690000895CF93C82F0E943D028C2F0E94460BC5
:1016A000CF9108950E94811C0C94490B0E94811CCB
:1016B0009091B901891721F08093B9010C94490BDD
:1016C0000895CF93DF93CDB7DEB72B970FB6F8947D
:1016D000DEBF0FBECDBF4F83588769877A878B8760
:1016E00061110E94DB149E012F5F3F4F86E0F901DC
:1016F00011928A95E9F785E0FE013796D9010190AC
:101700000D928A95E1F789819A814C815D81452B03
:1017100031F09F3F31F491E08F3F19F403C091E025
:1017200001C090E090FF09C049815A816B817C81A2
:101730008D819E810E94FC1305C0C9010E94640A2C
:101740008111F2CF2B960FB6F894DEBF0FBECDBF3E
:10175000DF91CF910895FC01808191810E94571102
:101760000895CF93882309F49CC0C82F8238C1F410
:101770000E94811C81FD95C069E3809132019091A6
:1017800033010E94691D0E94FD142FEF81EE94E049
:10179000215080409040E1F700C0000069E319C08B
:1017A000833801F50E94811C80FD7BC063E5809138
:1017B0003201909133010E94691D0E94FD142FEFA8
:1017C00081EE94E0215080409040E1F700C000009D
:1017D00063E580913201909133010E94741DCF9195
:1017E0000C94FD148438C1F40E94811C82FD59C000
:1017F00067E480913201909133010E94691D0E943B
:10180000FD142FEF81EE94E0215080409040E1F7ED
:1018100000C0000067E4DDCF8CEF8C0F813AD0F47C
:101820006C2F80913201909133010E94E91C882332
:1018300049F06C2F80913201909133010E94741D08
:101840000E94FD146C2F80913201909133010E940F
:10185000691DC5CF80E28C0F883048F4C77081E0E5
:1018600001C0880FCA95EAF70E94BE14B8CFEBE515
:10187000EC0FE33040F4F0E0E159FE4F808190E05E
:10188000CF910C94A71CC85AC73158F4EC2FF0E044
:10189000EE0FFF1FEF5BFE4F80819181CF910C9483
:1018A000BD1CCF910895882309F45BC0682F82384E
:1018B00079F40E94811C81FF54C069E38091320158
:1018C000909133010E94691D0E94FD1469E310C0CC
:1018D0008338B1F40E94811C80FF43C063E580918E
:1018E0003201909133010E94691D0E94FD1463E54D
:1018F00080913201909133010E94741D0C94FD146B
:10190000843879F40E94811C82FF2BC067E48091A7
:101910003201909133010E94691D0E94FD1467E419
:10192000E7CF8CEF860F813A18F380E2860F88307C
:1019300048F4677081E001C0880F6A95EAF70E9459
:10194000C414DCCF8BE5860F833020F480E090E078
:101950000C94A71C685A673120F480E090E00C9446
:10196000BD1C08951F93CF93DF93182FEB010E94A6
:10197000B10B209741F08FE99FE00197F1F700C08C
:1019800000002197F6CF812FDF91CF911F910C940A
:10199000530C893319F060E070E002C060E570E03C
:1019A0000C94B20C882321F00E94BE140C94FD14F8
:1019B0000895882321F00E94C4140C94FD14089506
:1019C000CF92DF92EF92FF920F931F93CF93DF930B
:1019D0007C01D62FC72FFC011281058102950F7063
:1019E0000E94B4148823B9F01123A9F08C2F807FB2
:1019F000803421F080E28D0F883068F08091AE0253
:101A000082FD09C082E00E945D150E94B41491E03D
:101A1000D82ED92601C0D12CCC2EC2948FE0C8225A
:101A20008C2D90E08C30910508F0C4C1FC01E15987
:101A3000FF4F0C9452258C2F807FCF70882311F09C
:101A4000C295C07F112399F0CC2309F49FC180E295
:101A50008D0F883010F0D11104C08C2F0E94BE145D
:101A600003C08C2F0E94CE140E94FD148FC18D2FB5
:101A70000E94530CCC2309F49DC180E28D0F883065
:101A800038F1DD2329F18C2F0E94D41424C08C2F2F
:101A9000807FCF70803211F0C295C07FDD2319F0B6
:101AA000D130A1F13DC08091AE0282FF17C0112359
:101AB00049F0CC2329F08C2F0E94BE140E94FD1403
:101AC00080E065C180E00E94530CCC2309F472C110
:101AD0008C2F0E94C4140E94FD146CC1112371F05C
:101AE000002341F0013031F40E94DE148C2B0E945F
:101AF000E61460C10E94DE148C2B1DC0002319F077
:101B0000013009F457C10E94F31425C0112321F0BC
:101B1000063008F04FC10EC0053008F04BC11BC0A5
:101B2000112361F0002331F0F701858180FF2EC180
:101B30008F7085838C2F0E94D20C3CC1002359F0FA
:101B4000D93309F034C1FFEF07EE13E0F150004044
:101B50001040E1F72AC18C2F0E94D90C2BC18C2F89
:101B600086958695837019F0813061F023C1112329
:101B700021F08D2F9C2F937002C080E090E00E9496
:101B8000A71C20C1112321F08D2F9C2F937002C020
:101B900080E090E00E94BD1C15C18C2F837009F07D
:101BA00047C011110BC12D2F229526952770220FAA
:101BB000220F6D2F6F70862F90E0A0E0B0E0022E14
:101BC00004C0880F991FAA1FBB1F0A94D2F7D4FF25
:101BD00010C04FE050E060E070E004C0440F551FBB
:101BE000661F771F2A95D2F740955095609570959E
:101BF00003C040E050E0BA01C695C695C3708A01A3
:101C00009B01082B192B2A2B3B2BC901B801C23091
:101C100049F058F4C13019F00E94D20FCFC00E9491
:101C2000C00FCCC00E94E40FC9C00E94BE0FC6C046
:101C3000112319F08C2F817001C08695882309F437
:101C4000BDC02D2F229526952770220F220F6D2FB4
:101C50006F70862F90E0A0E0B0E0022E04C0880FE5
:101C6000991FAA1FBB1F0A94D2F7D4FF10C04FE0E0
:101C700050E060E070E004C0440F551F661F771FFE
:101C80002A95D2F7409550956095709503C040E035
:101C900050E0BA01C695C695C3708A019B01082B16
:101CA000192B2A2B3B2BC901B801C23049F058F43B
:101CB000C13019F00E94971081C00E9485107EC02B
:101CC0000E94A9107BC00E94F80F78C0CF7011232A
:101CD00039F08C2F0E941E108D2F0E94D20C6EC0E6
:101CE0008D2F0E94D90C8C2F0E943F1067C0D23FCD
:101CF00021F128F4D03F41F0D13FC1F043C0D33FA0
:101D000019F1D43F79F03EC0112341F0053008F0BD
:101D100051C08C2F8F710E9464104CC0063008F0A7
:101D200049C0F7CF8091AE0282FF18C0112339F06D
:101D30008C2F8F710E941E103DC01123C9F38C2F70
:101D40008F710E943F1036C0112329F08C2F8F71A4
:101D50000E9409102FC00E9404102CC0112349F0CA
:101D6000CF718C2F0E941E1063E08C2F0E944215B1
:101D700021C081E00E945D150230E0F082E00E9407
:101D80005D1518C0112331F0002391F28D2F0E94B0
:101D9000B10B10C0002399F2D93349F41FEF27EE9D
:101DA00033E0115020403040E1F700C000008D2F9B
:101DB0000E94530C88EF8C0D843020F40E94811C0B
:101DC0000E94490BDD20C9F00E94B01480FD15C0AF
:101DD000F70112820E94AA140E941E10C7010E94DD
:101DE0001E0F0E94AA14DF91CF911F910F91FF90B7
:101DF000EF90DF90CF900C943F10DF91CF911F9127
:101E00000F91FF90EF90DF90CF9008950F931F9365
:101E1000CF93DF93EC01688179818A810E946211FE
:101E20008C010E94BB100E94AC0FB801CE010E9431
:101E3000E00CDF91CF911F910F910895CF93DF9325
:101E4000EC01988189812B813C81232B31F08F3FDC
:101E500031F481E09F3F19F403C081E001C080E0CC
:101E600080FD1DC0CE010E94EB0A811110C00E94AE
:101E7000B4148823A1F08A81882389F08091AE026E
:101E800082FD0DC082E0DF91CF910C945D15CE01F3
:101E90000E94060FCE01DF91CF910C94660ADF916C
:101EA000CF91089580E090E00E94A71C80E090E030
:101EB0000E94BD1C0E94DB140C94FD148091320121
:101EC000909133010E947F1D0C94520F0E94CB14FD
:101ED0000C945E0F92959F70963079F010F49250AA
:101EE00001C09A50923068F4803F69F018F4883E3F
:101EF00040F409C0843F29F406C0883E20F0813FA9
:101F000011F080E0089581E00895FC0180819181C5
:101F10000E9457110E946A0F0895CF93DF9300D05B
:101F200000D01F92CDB7DEB70F900F900F900F909B
:101F30000F90DF91CF910895CF93DF9300D000D021
:101F400000D0CDB7DEB726960FB6F894DEBF0FBE31
:101F5000CDBFDF91CF910895089508950C94AD0FF2
:101F60000C94AE0F0E94B00F6093C4017093C50132
:101F70008093C6019093C7010C94520F0C94B20F3A
:101F80000F931F930091C4011091C5012091C601C8
:101F90003091C701602B712B822B932B1F910F91D6
:101FA0000C94B20F0F931F930091C4011091C501BF
:101FB0002091C6013091C7016023712382239323AE
:101FC0001F910F910C94B20F0F931F930091C401B6
:101FD0001091C5012091C6013091C701602771277A
:101FE000822793271F910F910C94B20F0C94AD0F81
:101FF0000E94F60F6093C0017093C1018093C201EB
:102000009093C3010C94520F60E070E0CB010C94EC
:10201000F80F0F931F9341E050E060E070E08A01F9
:102020009B0104C0000F111F221F331F8A95D2F796
:10203000C901B8011F910F910C94F80F0F931F93D2
:1020400041E050E060E070E004C0440F551F661F9F
:10205000771F8A95D2F78091C0019091C101A0911C
:10206000C201B091C3018A019B01082B192B2A2BB5
:102070003B2BC901B8011F910F910C94F80F0F93DE
:102080001F9341E050E060E070E004C0440F551F32
:10209000661F771F8A95D2F7409550956095709589
:1020A0008091C0019091C101A091C201B091C30182
:1020B0008A019B01082319232A233B23C901B80164
:1020C0001F910F910C94F80F0F931F9341E050E074
:1020D00060E070E004C0440F551F661F771F8A95AB
:1020E000D2F78091C0019091C101A091C201B0913D
:1020F000C3018A019B01082719272A273B27C90109
:10210000B8011F910F910C94F80F0F931F9300913A
:10211000C0011091C1012091C2013091C301602B17
:10212000712B822B932B1F910F910C94F80F0F930F
:102130001F930091C0011091C1012091C201309103
:10214000C30160237123822393231F910F910C9469
:10215000F80F0F931F930091C0011091C1012091BE
:10216000C2013091C30160277127822793271F91F5
:102170000F910C94F80F0895292F220F920F990FA9
:10218000890FE82FE695E695E695877051E001C046
:10219000550F8A95EAF785E0E89FF0011124E55490
:1021A000FE4F20E030E070E04081CB01022E02C003
:1021B000969587950A94E2F7817081958427852307
:1021C000842781932F5F3F4F2530310569F70895AC
:1021D000292F220F920F990F890F682F6695669508
:1021E0006695982F977085E0689FB001112440E0B4
:1021F00050E080E0FB01E40FF51FE554FE4F208125
:1022000030E0092E02C0369527950A94E2F7217036
:102210003327042E01C0220F0A94EAF7822B4F5F66
:102220005F4F4530510531F70895BF92CF92DF924D
:10223000EF92FF920F931F93CF93DF938C01C09087
:10224000C001D090C101E090C201F090C301809123
:10225000C4019091C501A091C601B091C701C82ADF
:10226000D92AEA2AFB2ACFE1D0E0D701C6010C2EF9
:1022700004C0B695A795979587950A94D2F780FDE7
:1022800004C0219790F7B12C07C0BC2EB8018C2F49
:102290000E941D180197A9F38B2DDF91CF911F91FB
:1022A0000F91FF90EF90DF90CF90BF900895CF9364
:1022B000DF93EC010E941511BE010E941D18DF91F1
:1022C000CF9108951F93CF93DF93EB019091BA01C3
:1022D000992321F0CB010E94571113C0882349F0A4
:1022E000CB010E941511182F682FCE010E94BC103F
:1022F00004C0CB010E94E810182FBE01812F0E945C
:102300001D18DF91CF911F9108951F93CF93DF93F5
:10231000C091C80116E08091C901C81799F0D0E0BA
:102320001C9FF0011D9FF00D1124E653FE4F4081CC
:10233000518162817381848195810E949C0F2196D5
:10234000C770E9CFDF91CF911F9108954091FA01B5
:102350005091FB016091FC017091FD018091FE01A3
:102360009091FF010C949C0FEF92FF920F931F939B
:10237000CF93DF938091FF0182958F7009F065C044
:102380008091FC01882309F460C08091C801F0901D
:10239000C9011091FA010091FB016091FD0170915A
:1023A000FE0191E01F3F09F090E0C0913001D09113
:1023B0003101292F96E0E92E8F1509F446C06115E9
:1023C000710521F00F3F21F030E003C031E001C082
:1023D000322F90E030FD36C0E89EF001E99EF00D0E
:1023E0001124DF01A653BE4F11963C911197301373
:1023F00029C03C91311326C012963C91129731119D
:1024000021C013964D915C911497461B570B4C17A6
:102410005D07C0F48091FF018F7080618093FF01A0
:10242000E153FE4F80818F70806180838AEF91E05D
:102430000E941E0FDF91CF911F910F91FF90EF909F
:102440000C94851101968770B7CFDF91CF911F91C2
:102450000F91FF90EF9008959F92AF92BF92CF920D
:10246000DF92EF92FF920F931F93CF93DF93CDB73D
:10247000DEB761970FB6F894DEBF0FBECDBF8C01FB
:1024800085E0F801DE011D9601900D928A95E1F735
:10249000D8011296EC909091FA01E091FB01209105
:1024A000FD013091FE012115310531F0EF3F31F48E
:1024B00081E09F3F19F403C081E001C080E0B82FA4
:1024C000B1709B2E80FD47C1D8014C9111965C9153
:1024D00011971396AD90BC9014978AEFC82E81E0A7
:1024E000D82EF090FC01B501621B730B20913001D6
:1024F00030913101FF2009F4D9C08091FF016217AA
:10250000730708F095C0282F207F09F052C05E1392
:1025100013C0491311C0FE2CE1100EC08F708061F2
:102520008093FF010E94A611C6010E941E0F809198
:10253000FF01F80185834DC1AB2831F05F3F31F4D5
:1025400081E04F3F19F403C081E001C080E080FDCD
:1025500003C081E08E2502C080E090E0F82FF1708A
:10256000FF2E80FF1CC08091C8012091C90136E078
:10257000821709F40BC190E0389FF001399FF00DEC
:102580001124E653FE4F6181561306C06081461345
:1025900003C06281E61203C001968770E9CFFE2C6A
:1025A000EE2009F416C18091FF0181608093FF0144
:1025B00054C05E1306C0491304C0E11002C0F80104
:1025C00099C0C8010E94850F882361F1EE2051F166
:1025D0002091FF01822F82958F7090E0029774F016
:1025E0008091FA019091FB0198878F831986BB86B1
:1025F000AA862C87CE0107960E941E0F86E0F8015E
:10260000AAEFB1E001900D928A95E1F70E94B41112
:102610000E94A6110AC05E1711F1C8010E94850F21
:1026200081112CC0C8010E941E0FFF24F394D1C059
:10263000282F207F81F77A2DB98AA88A6E2D898963
:102640000E948D0F8AEF91E00E941E0F86E0D60156
:102650001D928A95E9F70E94A611F12CBAC0491380
:10266000DCCFE110DACFF8018583C8010E941E0F8C
:1026700086E0D6011D928A95E9F7ABC0EE2091F273
:102680002091FF01822F82958F7090E002970CF4C9
:10269000B5CF8091FA019091FB019A8389831B82C7
:1026A000BD82AC822E83CE010196A6CF621773073E
:1026B00008F044C0FE2CEE2009F4B4CF5E1330C005
:1026C00049132EC02091FF0120FD21C0822F829549
:1026D0008F70482F50E041155105C9F0F80125834E
:1026E0004F30510541F08F5F982F9295907F822F48
:1026F0008F70892B8583C8010E941E0F86E0F80128
:10270000AAEFB1E001900D928A95E1F73CC086E016
:10271000F801AAEFB1E001900D928A95E1F759C056
:10272000C8010E94850F811169CF8091FF018160EE
:102730008093FF01C8010E941E0F4BC07A2DB98AF9
:10274000A88A6E2D89890E948D0F86E0D6011D9280
:102750008A95E9F718C0EE2009F464CFC8010E94F9
:10276000850FF82E882309F45DCF86E0F801AAEFE3
:10277000B1E001900D928A95E1F78AEF91E00E9415
:10278000AB0B0E94B4110E94A61123C04D875E8737
:102790008D859E850E945711292F22952F702230FA
:1027A00028F49F7039F0811105C00BC0243028F443
:1027B0009F7049F4805E883020F0C8010E941E0F8F
:1027C0009F2CF92C06C0D80115969C91907F91F70B
:1027D000F8CF8F2D61960FB6F894DEBF0FBECDBF38
:1027E000DF91CF911F910F91FF90EF90DF90CF90ED
:1027F000BF90AF909F9008951F93CF93DF93CDB775
:10280000DEB72C970FB6F894DEBF0FBECDBF4F8357
:10281000588769877A878B879C87CE0107960E94A5
:102820002C128823D1F09F8188852A853B85232B14
:1028300031F08F3F31F481E09F3F19F403C081E014
:1028400001C080E080FD47C04F81588569857A8549
:102850008B859C850E949C0F3EC086E0FE013796CA
:10286000DE01119601900D928A95E1F7FF81E885CE
:102870006A857B856115710531F0EF3F31F481E0A8
:10288000FF3F19F403C081E001C080E080FD23C058
:102890002091C90130E0C9010196877099274091C4
:1028A000C80150E084179507F1F1F983EA837D832D
:1028B0006C8396E0929FD001939FB00D1124A65394
:1028C000BE4FFE01319601900D929A95E1F78093EB
:1028D000C9010E94851116E08091C8019091C9013B
:1028E000891771F1189FC001112486539E4F0E94D1
:1028F0002C12882329F1E091C8011E9FF0011124B8
:10290000E653FE4F408151816281738184819581BC
:102910000E949C0F8091C80190E0019687709927D2
:102920008093C801D9CF0E94660F1092C9011092FE
:10293000C801EAEFF1E086E0DF011D928A95E9F730
:102940002C960FB6F894DEBF0FBECDBFDF91CF91AE
:102950001F9108958091200285958595859508950C
:10296000809120028770089590912002977081E0F5
:1029700009F480E008958091430208959091430204
:10298000892B809343020895809590914302892377
:102990008093430208951092430208959091420259
:1029A000892B809342020895809590914202892359
:1029B000809342020895109242020895809121026C
:1029C000089508950C94E1140C94E2149091AE02D1
:1029D00092FD08C090912102981721F08093210266
:1029E0000C94E414089580912102882329F0109218
:1029F000210280E00C94E4140895CF93DF93E091DA
:102A00003201F0913301809143028083E0913201E1
:102A1000F0913301908180914202892B80838091D3
:102A20002102882381F0E0913201F09133019081FD
:102A3000892B808380913201909133010E94D31CB5
:102A400081110E94F314C0913201D091330140E210
:102A500050E060E072E0CE010E94B425892B69F05D
:102A600080E2FE01A0E0B2E001900D928A95E1F7CC
:102A7000CE01DF91CF910C948D1CDF91CF91089501
:102A80000C94E1149091AE0292FD10C098E0899FE1
:102A900090011124262B209320020E941E10809169
:102AA00020028595859585950C9440150C941E10F3
:102AB0001092200280E00C94401520912002809515
:102AC000822380932002982F977099F430E0482F4A
:102AD000082E000C550B2417350759F09091AE02C3
:102AE00092FD07C08595859585950E943F100C94B1
:102AF000581508959091AE0292FB222720F92817CD
:102B000069F080FB92F99093AE028091AD029091B2
:102B1000AE020E94C81582E00C945D150895809164
:102B2000AE0282FB882780F991E089270C947A1500
:102B300081E00C947A1580E00C947A156FEF7FEFAA
:102B400080E090E00C940D2680E090E00E94D92572
:102B500021E0893E9E4F09F020E0822F089582E017
:102B600090E00C94D12583E090E00C94D125CF9394
:102B700084E090E00E94D125C82F82E290E00E947C
:102B8000D1252C2F30E0A901582BCA01CF910895EF
:102B9000CF93C92F682F84E090E00E94EF256C2F1F
:102BA00082E290E0CF910C94EF25AB01BC018FE065
:102BB00090E00C940126AB01BC0183E190E00C9401
:102BC000012660E070E0CB010C94DB1560E070E062
:102BD000CB010E94D5150C94E11569EE7EEF80E0E3
:102BE00090E00E940D2660E082E090E00E94EF25D8
:102BF00060E083E090E00E94EF251092C401109203
:102C0000C5011092C6011092C70160E084E090E017
:102C10000E94EF2560E082E290E00E94EF2560E0F4
:102C200085E090E00E94EF2560E086E090E00E9461
:102C3000EF256FEF87E090E00E94EF2540E050E045
:102C4000BA0188E090E00E94012660E08DE090E00B
:102C50000E94EF2540E050E0BA0188E190E00E9438
:102C6000012660E087E190E00E94EF2540E050E01F
:102C7000BA018CE190E00E94012660E070E080E201
:102C800090E00E940D2640E050E0BA0188E190E01B
:102C90000E9401260C94E6150C94ED15682F8EE029
:102CA00090E00C94EF250E94E01D60934902709320
:102CB0004A0280934B0290934C02609345027093BA
:102CC00046028093470290934802089585B7806832
:102CD00085BF85B7806885BF089581E008950C940D
:102CE0006D1608950C9471160C9471160C9474164C
:102CF0000C9471160C9478160C9471160E9466163A
:102D000089EF98E10E94771C0E947C160C947A1639
:102D10000E9472160C9471160E9413190C94480BA1
:102D20000E94CB1D0E94B8190E948C160C94761636
:102D3000DF92EF92FF920F931F93CF93DF93CDB764
:102D4000DEB72A970FB6F894DEBF0FBECDBF0E9444
:102D5000C319D82E81110E94531680E00E943719A2
:102D6000F82EE0904402E82689F48FEF89838A8365
:102D70001B820E94D41D8160782F9D838C834981A2
:102D80005A816B818D810E94610B2CC080914D0214
:102D900081FD0E943D1900E011E08E2D8123E9F0B4
:102DA0000E946F16882399F00E831F82F12281E022
:102DB00009F480E088870E94D41D8160782F9A876B
:102DC00089874E815F8168858A850E94610B809129
:102DD000440218271093440205C00F5F110F0630FC
:102DE000E1F6C3CF81E0D11001C080E02A960FB692
:102DF000F894DEBF0FBECDBFDF91CF911F910F9131
:102E0000FF90EF90DF9008950E9498160C94560B57
:102E1000CF93DF930E942218EC01811522E59207DF
:102E2000E8F5811531E5930708F0B6C0883E9105B5
:102E300028F5803E910508F0E9C0883A910570F4C4
:102E4000853A910508F07AC08130910509F473C084
:102E500008F4D9C0049708F0D9C0D5C08F3B9105BC
:102E600008F0D1C0C85AD0E0CC0FDD1FCE58DE4FDD
:102E70000990D881C02DCE019464C9C0811540E568
:102E8000940708F069C0811550E4950708F060C008
:102E90009A9581159F4108F4B9C0B5C0811536E5F2
:102EA000930728F5811545E5940708F092C0811530
:102EB00054E5950708F087C0AC0143705527282FCB
:102EC00026952695C115D34508F06CC081E090E0A9
:102ED00002C0880F991F4A95E2F740E2249F9001B3
:102EE0001124EC01C22BD32BCE019C6890C081151C
:102EF0002AE5920780F4811539E5930708F072C03E
:102F0000811548E5940708F47EC0D82FCC27CE0160
:102F1000806F906A7CC090568115904208F073C013
:102F20008D2F8F710E94B618DD27D0628F71AE0190
:102F3000582BCA016CC081E090E069C0C55AD0E04E
:102F4000C056DE4F8881C82FD0E0CE0190645FC0AC
:102F5000DF70CE01906A5BC074E0969587957A9594
:102F6000E1F7282F23703C2F337081E090E002C0FE
:102F7000880F991F3A95E2F79C68AC01522B9A0191
:102F80009C2F9F709695969550E2959FE001112495
:102F9000C9018C2B9D2B3BC0D82FCC27CE01816F34
:102FA000906A35C081E090E002C0880F991F4A9571
:102FB000E2F750E2259F90011124EC01C22BD32BA4
:102FC000CE019A6824C0D82FCC27CE01846F906A96
:102FD0001EC00E94B6188F7190E0D82FCC27CE016A
:102FE000906215C08F700E94B61894E0D695C79570
:102FF0009A95E1F7CF70D0E0DC2FCC27D0699E0105
:10300000282BC90104C080E090E001C0CE01DF910F
:10301000CF910895272F30E0280F311D86E0829F41
:10302000F001839FF00D1124E60FF11DEE0FFF1F3D
:10303000E85DFE4F8591949108950E940A180E94C0
:10304000081708958238910569F1B0F4813391052C
:1030500009F46DC048F48932910509F463C08A32DD
:10306000910509F469C008958533910509F455C0A7
:1030700089339105B9F00895833E910569F138F4DB
:10308000803E9105B1F0823E910509F10895863E9A
:103090009105A9F1873E9105B9F1843E910509F0AA
:1030A00064C023C02091AD0220FD4FC021FD4DC062
:1030B00008958091AD0280FD44C08091AE0280FFF2
:1030C00044C08091AD0284FD42C083EE4DC080912A
:1030D000AD0282FF38C0F5CF8091AD0282FD33C0D2
:1030E0008091AE0280FD31C0ECCF8091AE0281FFB5
:1030F00032C08091AD0284FD2AC087EE35C0809138
:10310000AD0283FF26C0F5CF8091AD0283FD21C0C3
:103110008091AE0281FD1FC0ECCF8091AD0285FD94
:103120001CC01DC08091AD0285FD19C016C08091E4
:10313000AD0286FD16C017C08091AD0286FD13C09A
:1031400010C089E311C082EE0FC080EE0DC080E098
:103150000BC086EE09C084EE07C089E205C085E396
:1031600003C08AE201C081E390E008959091AD022E
:1031700092FF0DC0282F2871283019F4877F8460B2
:1031800006C0282F2471243011F48B7F886093FFB0
:103190000DC0282F2871283119F4877E846106C05C
:1031A000282F2471243111F48B7E88612091AE0286
:1031B00020FF0DC0382F3871383019F4877F8160B7
:1031C00006C0382F3171313011F48E7F886021FFB5
:1031D0000DC0282F2871283119F4877E816106C01F
:1031E000282F2171213111F48E7E886194FD877E14
:1031F000089580E008950C949E150E94C3198FE3F2
:103200009CE90197F1F700C000000E94C31980E01B
:103210000E94371980FF04C00E94FB180C94211EE5
:1032200008950C94FD180E94A415811102C00E94FB
:103230004C160E94AF1580934D020E94B7159093D3
:10324000AE028093AD020E9411190E94B315682F3F
:1032500070E080E090E00E94BE0F6091C00170912C
:10326000C1018091C2019091C3010C94F60FE82F27
:10327000F0E0E055FD4F80810895089580EA8A9539
:10328000F1F7089500C008950C943E1908950C9428
:1032900046190C944619F894E82FE295EF70F0E087
:1032A00031A1282F2F7081E090E001C0880F2A956E
:1032B000EAF7982F9095932391A392A1892B82A34B
:1032C000789408950F931F93CF93DF9386EC0E9419
:1032D0004B19C3EAD1E009EA11E089918F3F11F05F
:1032E0000E944B190C171D07C1F7DF91CF911F9159
:1032F0000F9108950F931F93CF93DF938C01D62FD7
:10330000F8946E9A769878940E944219E3EAF1E074
:1033100031E0C0E021912F3F89F0A22FA295AF703C
:10332000B0E090968C9190E02F7002C095958795B3
:103330002A95E2F780FD02C0832F01C080E0C82BF0
:10334000330F81E0E93AF80729F786EC0E944B1920
:1033500061E0C11101C060E08D2F0E944419F801A5
:10336000ED0FF11DC083DF91CF911F910F91089553
:103370000E9462191092B0021092AF0281E00E9486
:10338000E9190C94D70A1F93CF93DF931F92CDB7FF
:10339000DEB7198260E0CE0101960E947A19909101
:1033A000AF02898111E0981301C010E09813809357
:1033B000AF02212F41E060EB72E08FEA92E00E94C1
:1033C000EA190E94D90A812F0F90DF91CF911F91A6
:1033D00008950895FF920F931F93CF93DF938C016D
:1033E000F62ED72FC42F222349F081E0809350027C
:1033F0000E94D41D90934F0280934E028091500200
:103400008823C1F080914E0290914F020E94EC1DE2
:10341000059780F0EF2DFD2FD8014C2F50E0CD0106
:10342000801B910B841795071CF48D918193F7CF26
:1034300010925002DF91CF911F910F91FF9008954C
:103440000E94CE1F0E9490160C94DA1F0E94DE1F6D
:103450000E9404170C94F81F0E94BF1D0E94B51F04
:103460000E947E160E94201A0E94261A0E94881628
:10347000FBCFCF93DF93EC01FB018281882309F41A
:103480003CC1C430FDE5DF0760F4CB3F9CE5D907C4
:1034900088F49E0122503C452431310508F02EC1AC
:1034A00009C0C236EDE5DE0729F0C63AFDE5DF07C3
:1034B00009F024C10E94B7159093AE028093AD022B
:1034C000C1318CE5D80709F4C6C008F042C0C93044
:1034D000ECE5DE0709F49BC000F5C5308CE5D807A4
:1034E00009F485C078F4C330ECE5DE0709F478C050
:1034F00008F07AC0C230DC4509F0F5C08091AD0219
:103500008160EFC0C7309CE5D90709F478C008F0A6
:103510007AC08091AD028061E4C0CD30FCE5DF0768
:1035200009F487C058F4CB309CE5D90709F479C079
:1035300008F07BC08091AD0288606FC0CF30FCE5A1
:10354000DF0709F480C008F082C08091AD02877F58
:10355000C8C0CE3F9CE5D90709F471C000F5C5315C
:10356000FCE5DF0709F485C068F4C3319CE5D907A1
:1035700009F475C008F095C00E94660F8091AD02F5
:103580008F77AFC0CC3FFCE5DF07A9F108F054C04E
:10359000CB3FDC4509F0A7C08091AE0240C0C230ED
:1035A000EDE5DE0709F489C058F4C1158DE5D807AB
:1035B00009F45AC008F069C08091AE0282602FC041
:1035C000C236EDE5DE0709F47CC0C63AFDE5DF074B
:1035D00009F481C0C330DD4509F085C080E06EC0CC
:1035E0008091AD0282607DC08091AD0216C0809155
:1035F000AD02886076C08091AE0282604FC080913B
:10360000AD0280626EC08091AD0280646AC00E948B
:10361000660F8091AD02806864C0846062C0816082
:103620003DC08091AD028E7F5CC08091AD028D7FE8
:1036300058C08091AD0216C08091AE0218C0809132
:10364000AE028D7F2BC08091AD028F7E4AC08091EB
:10365000AD028F7D46C08091AD028F7B42C08091CC
:10366000AD02877F8B7F3DC08091AE028D7F8E7FC4
:1036700015C08091AD0282FB222720F991E09227AC
:1036800090FB82F990FB83F92CC08091AE02982FB9
:10369000909591708E7F892B90FB81F98093AE027B
:1036A00022C00E94660F8091AD0287FB222720F97D
:1036B00091E0922790FB87F914C081E00E944E169A
:1036C00012C08091AD0284FB222720F991E092275D
:1036D00090FB84F906C08091AD02982F909590FBE5
:1036E00080F98093AD028091AD029091AE020E946C
:1036F000C8150E94660F80E001C081E0DF91CF9184
:103700000895CF93DF9386319C4541F5EB010E94EC
:10371000BB14982F8A812091320130913301882384
:1037200079F09A7A81E009F480E080935102911156
:1037300002C069E201C065E3C9010E94691D0AC0B7
:1037400080915102811102C069E201C065E3C901A3
:103750000E94741D0E94FD1480E001C081E0DF9191
:10376000CF9108950F931F93CF93DF93C42FD22F40
:10377000FC0182818823C9F0409354020E94D41D29
:10378000909353028093520280E28C0F883008F0AD
:1037900057C0C77081E001C0880FCA95EAF7DF9172
:1037A000CF911F910F910C94D20C80915402481329
:1037B00030C080915202909153020E94EC1D883CCF
:1037C000910538F510E21D0FCD17B9F080E28C0F8E
:1037D000883040F4C77081E001C0880FCA95EAF7CD
:1037E0000E94D90C183028F581E09D2F977001C0F8
:1037F000880F9A95EAF70E94D20C802F0E94C90C7C
:103800001830F0F4D77081E001C0880FDA95EAF73C
:103810000AC080E28C0F883098F4C77081E001C044
:10382000880FCA95EAF7DF91CF911F910F910C9401
:10383000D90C802FDF91CF911F910F910C94C90C5F
:10384000DF91CF911F910F9108950F939C01CB01B0
:10385000243F4CE5340731F188F4293DFCE53F076E
:10386000D9F02A3D4CE5340779F1283D3C45A9F5CE
:1038700006E221EE41EE68ED7CE52BC0263FFCE53B
:103880003F07E1F0A8F0273F3C4539F507E225EE78
:1038900046EE67EF7CE51DC007E225EE45EE69EDDB
:1038A0007CE517C006E221EE40EE64EF7CE511C036
:1038B00007E225EE44EE65EF7CE50BC006E221EE63
:1038C00042EE66EF7CE505C008E221E045EE6AEDD8
:1038D0007CE50E94B21B80E008C0FC018281882345
:1038E00019F01092540201C081E00F910895909355
:1038F000AB018093AA01089590935A0280935902D4
:103900000895E0915902F0915A02309721F0019008
:10391000F081E02D099480E00895E0915902F09142
:103920005A02309799F020914001222359F02091BA
:10393000AD0227FF07C0DC012C9111962C93119743
:1039400026E02C930280F381E02D099408952091C4
:103950005702309158022817390771F09093580296
:1039600080935702E0915902F0915A02309721F06A
:103970000680F781E02D0994089520915502309139
:1039800056022817390771F090935602809355021A
:10399000E0915902F0915A02309721F00084F185AC
:1039A000E02D09940895FC0132968091400188230E
:1039B00031F08091AD0287FF02C09EE101C096E028
:1039C00080E0915028F021912223D9F38F5FF9CF25
:1039D0000895662351F1209140012223E9F02091BE
:1039E000AD0227FF19C0462F4695469546954E31A4
:1039F000E0F4677021E030E002C0220F331F6A95C7
:103A0000E2F7FC01E40FF11D828190E028233923C5
:103A100081E0232B69F409C0FC01329608962191BC
:103A2000621729F0E817F907D1F780E0089581E0DF
:103A300008959C01FC0132969FEF80E0419146176A
:103A400089F09F3F19F4411101C0982F8F5F863094
:103A5000A9F79F3F39F0F901E90FF11D97FDFA959C
:103A60006283089508959C012A5F3F4FFC014281C3
:103A7000461301C01282019682179307B9F7089581
:103A8000262F2695269526952E3168F4FC01E20F07
:103A9000F11D677021E030E001C0220F6A95EAF75E
:103AA0008281282B22830895262F269526952695F8
:103AB0002E3170F4FC01E20FF11D677021E030E05F
:103AC00001C0220F6A95EAF720958281282322837C
:103AD000089520914001222329F02091AD0227FD75
:103AE0000C94401D0C94191D20914001222329F0B3
:103AF0002091AD0227FD0C94541D0C94331D209190
:103B00004001FC013296222331F08091AD0287FF03
:103B100002C08EE101C086E0DF011D928A95E9F7BF
:103B2000089508950C94911D83E080935B020C949A
:103B3000921D811102C081E001C082E080935B028E
:103B40000C94921D0C94991D81E080935B020C945F
:103B5000921D0C94A41D08950C94AB1D0C94AB1DE8
:103B60000E94AE1D0E94C3190E94AC1D80E00E94FD
:103B7000371991E0811101C090E0892F08950895CF
:103B80008091B902843011F00C943D0B08950E948D
:103B9000660F0C943F0B82E084BD93E095BD9AEFD5
:103BA00097BD80936E0008952FB7F8948091B1026D
:103BB0009091B202A091B302B091B4022FBF0895C8
:103BC0002FB7F8946091B1027091B2028091B30264
:103BD0009091B4022FBF08959C014FB7F894809143
:103BE000B1029091B202A091B302B091B4024FBF62
:103BF000821B930B089578941F920F920FB60F9229
:103C000011248F939F93AF93BF938091B1029091B2
:103C1000B202A091B302B091B4020196A11DB11DF0
:103C20008093B1029093B202A093B302B093B40216
:103C3000BF91AF919F918F910F900FBE0F901F90EA
:103C4000189581E08093E00080E28093D800109284
:103C5000C9008FE19EE40197F1F700C0000087E002
:103C600090EBDC018093C2029093C302A093C40244
:103C7000B093C5029CE088E10FB6F894A8958093B4
:103C800060000FBE90936000FFCF80917F02089587
:103C90000895CF93DF9320914001222339F02091A2
:103CA000AD0227FF03C060E222E002C068E021E02D
:103CB0002093E9002FEF3091E800215035FD06C038
:103CC00035ED3A95F1F700002111F5CF2091E8008C
:103CD00025FF1DC0EC0180914001811105C040E02D
:103CE00050E068E070E003C070E040E050E0CE01DA
:103CF0000E946A208091E8008E778093E80080E23D
:103D0000FE01AFE5B2E001900D928A95E1F7DF91F7
:103D1000CF91089580935C0270935E0260935D0280
:103D20008091B902843001F582E08093E9008FEF41
:103D30009091E800815095FD06C095ED9A95F1F7B8
:103D400000008111F5CF8091E80085FF0DC040E0B3
:103D500050E063E070E08CE592E00E946A20809180
:103D6000E8008E778093E8000895BC0184E00C940D
:103D70008A1EBC0183E00C948A1E08958091B802CB
:103D8000811109C00E94FB210E9458228091E2000B
:103D900084608093E20008951092B80208950C9414
:103DA000A91D6091B50281E0611101C080E00C9411
:103DB000941D9091B90281E0943009F080E0609107
:103DC000B5020C94991D42E061EC81E00E947421DF
:103DD00042E261EC82E00E9474219091B90281E09C
:103DE000943009F080E06091B5020C94A21D80919E
:103DF000BB02833009F461C030F4813071F082304D
:103E000009F49AC008958A3009F486C08B3009F409
:103E10006CC0893009F0A8C020C08091BA02813AF4
:103E200009F0A2C08091E800877F8093E80080912C
:103E3000BE029091BF02892B21F460E28FE592E0EF
:103E400003C060E080E090E070E00E94B5208091C7
:103E5000E8008B778093E80008958091BA02813260
:103E600009F082C08091BE029091BF02029708F0D3
:103E70007BC08091E800877F8093E8008091E80014
:103E800082FD05C08091B9028111F8CF6DC02091EB
:103E9000F3008091F20090E0922B029731F4809130
:103EA000F100813011F0863021F48091F10080938F
:103EB0007F028091E8008B7753C08091BA02813AEB
:103EC00009F052C08091BE029091BF02892B09F087
:103ED0004BC08091E800877F8093E8008091E800E4
:103EE00080FFFCCF8091400136C08091BA028132C0
:103EF000D9F58091BE029091BF02892BA9F58091DE
:103F0000E800877F8093E8000E94A9218091BC028D
:103F1000809340010C94660F8091BA02813221F5A2
:103F20008091E800877F8093E8000E94A92180911A
:103F3000BD028093800208958091BA02813AA1F473
:103F40008091E800877F8093E8008091E80080FFFF
:103F5000FCCF809180028093F1008091E8008E7701
:103F60008093E8000C94A921089584B7877F84BFCB
:103F70000FB6F894A89580916000886180936000E6
:103F8000109260000FBE90E080E80FB6F894809326
:103F90006100909361000FBE0C94A41D0E94FB2150
:103FA0000E945822E2EEF0E0808184608083789461
:103FB0000C94ED2484E391E00C947C1C8091B90274
:103FC0008530A9F48091B902853079F40E94C01D32
:103FD0008091B7028823B1F30E94B01D882391F32A
:103FE0000E9454200E94660FEDCF0C94C71D0895C7
:103FF00008950C94FB1F292F332723303105C9F076
:1040000060F42130310581F02230310509F044C0DF
:104010008BE390E026E932E043C021323105E1F044
:104020002232310549F138C082E190E021ED32E0E1
:1040300037C099278130910549F028F0029761F542
:10404000E8E5F2E005C0E2E9F2E002C0EAE7F2E00A
:10405000849190E09F0124C06115710541F06130A9
:104060007105D1F489E090E021EC32E019C089E0DB
:1040700090E028EA32E014C06115710541F061302A
:10408000710551F48DE690E023EE32E009C080E442
:1040900090E020E533E004C080E090E020E030E0F4
:1040A000FA0131832083089580E189BD82E189BDD1
:1040B00009B400FEFDCF8091D8008F7D8093D80099
:1040C0008091E00082608093E0008091E00081FDBB
:1040D000FCCF0895CF92DF92EF92FF920F931F9340
:1040E000CF93DF93EC018B017A010E94C8218111EB
:1040F00033C0E114F10439F0F70180819181081B8C
:10410000190BC80FD91FC12CD12C0115110519F19C
:104110008091E80085FD16C08091E8008E7780933D
:10412000E800E114F10449F0F70180819181C80EA3
:10413000D91ED182C08285E00FC00E94C821882389
:1041400021F30AC089918093F10001501109FFEF1A
:10415000CF1ADF0ADACF80E0DF91CF911F910F9164
:10416000FF90EF90DF90CF9008952091C0023091A2
:10417000C1022617370748F06115710539F42091FF
:10418000E8002E772093E80001C0B901FC0120E08F
:104190006115710579F18091B9028823F1F18530BB
:1041A000F1F18091E80083FD3CC08091E80082FD40
:1041B0002EC08091E80080FFEBCF2091F30080912A
:1041C000F20090E0922B6115710551F08830910555
:1041D00038F421912093F100615071090196F3CFD9
:1041E00021E0089709F020E08091E8008E77809325
:1041F000E800CECF2111CFCF0AC08091B902882329
:1042000061F0853061F08091E80083FD0AC0809103
:10421000E80082FFF2CF80E0089582E0089583E015
:10422000089581E008952091C0023091C1022617BF
:10423000370748F06115710539F42091E8002E77B1
:104240002093E80001C0B901FC0120E0611571056F
:1042500091F18091B902882309F440C0853009F4B6
:104260003FC08091E80083FD3DC08091E80082FD61
:104270002FC08091E80080FFE9CF2091F30080916A
:10428000F20090E0922B6115710559F0883091058C
:1042900040F424912093F100319661507109019608
:1042A000F2CF21E0089709F020E08091E8008E77B6
:1042B0008093E800CBCF2111CCCF0AC08091B90206
:1042C000882361F0853061F08091E80083FD0AC0A9
:1042D0008091E80082FFF2CF80E0089582E00895A7
:1042E00083E0089581E00895982F973068F59093C2
:1042F000E900981739F07091EC002091ED00509191
:10430000F00003C0242F762F50E021FD02C09F5FF4
:10431000ECCF3091EB003E7F3093EB003091ED001D
:104320003D7F3093ED003091EB0031603093EB0036
:104330007093EC002093ED005093F0002091EE007C
:1043400027FDE5CF80E008958F708093E90081E03C
:1043500008958091BA0287FF11C08091E80082FD24
:1043600005C08091B9028111F8CF11C08091E80099
:104370008B770BC08091B902882349F08091E800C7
:1043800080FFF8CF8091E8008E778093E800089551
:104390002091E4003091E50095E64091EC00842FF7
:1043A000817040FF23C08091E80080FD1DC0809196
:1043B000B902882399F0853099F08091EB0085FD52
:1043C00011C04091E4005091E5002417350729F30E
:1043D000915011F09A01E1CF84E0089582E00895B0
:1043E00083E0089581E0089580E008954091E80019
:1043F00042FFDDCF08950E9469220E947122E0EE03
:10440000F0E0808181608083E8EDF0E080818F774B
:10441000808319BCA7EDB0E08C918E7F8C93808156
:104420008F7E80831092B80208950F931F93CF93CD
:10443000DF930E9469220E947122C8EDD0E088813A
:104440008F77888388818068888388818F7D88833F
:1044500019BC1092B9021092B5021092B7021092D4
:10446000B60200EE10E0F80180818B7F80838881A6
:104470008160888342E060E080E00E947421E1EE88
:10448000F0E080818E7F8083E2EEF0E080818160C9
:104490008083808188608083F80180818E7F808323
:1044A000888180618883DF91CF911F910F9108955A
:1044B000E8EDF0E080818F7E8083E7EDF0E08081A1
:1044C0008160808384E082BF81E08093B8020C9495
:1044D0001522E8EDF0E080818E7F80831092E2006B
:1044E00008951092DA001092E10008951F920F9241
:1044F0000FB60F9211242F933F934F935F936F93B7
:104500007F938F939F93AF93BF93EF93FF9380918C
:10451000E10082FF0BC08091E20082FF07C0809122
:10452000E1008B7F8093E1000E94EC248091DA000F
:1045300080FF1FC08091D80080FF1BC08091DA00EF
:104540008E7F8093DA008091D90080FF0DC080E1DA
:1045500089BD82E189BD09B400FEFDCF81E0809371
:10456000B9020E94BE1E05C019BC1092B9020E9479
:10457000CC1E8091E10080FF19C08091E20080FF95
:1045800015C08091E2008E7F8093E2008091E2006E
:1045900080618093E2008091D80080628093D8008F
:1045A00019BC85E08093B9020E94D11E8091E10080
:1045B00084FF30C08091E20084FF2CC080E189BD7F
:1045C00082E189BD09B400FEFDCF8091D8008F7DC6
:1045D0008093D8008091E1008F7E8093E1008091EC
:1045E000E2008F7E8093E2008091E2008160809300
:1045F000E2008091B502882311F084E007C0809129
:10460000E30087FD02C081E001C083E08093B9022E
:104610000E94D91E8091E10083FF29C08091E200B1
:1046200083FF25C08091E100877F8093E10082E0D5
:104630008093B9021092B5028091E1008E7F809341
:10464000E1008091E2008E7F8093E2008091E200A1
:1046500080618093E20042E060E080E00E9474218B
:104660008091F00088608093F0000E94CF1EFF913F
:10467000EF91BF91AF919F918F917F916F915F91DA
:104680004F913F912F910F900FBE0F901F90189553
:104690001F920F920FB60F9211242F933F934F93B7
:1046A0005F936F937F938F939F93AF93BF93CF93BA
:1046B000DF93EF93FF93C091E900CF708091EC00FE
:1046C000D82FD17080FDD0E81092E9008091F000E1
:1046D000877F8093F00078940E948C231092E900E9
:1046E0008091F00088608093F000CD2BCF70C09354
:1046F000E900FF91EF91DF91CF91BF91AF919F9131
:104700008F917F916F915F914F913F912F910F907A
:104710000FBE0F901F9018951F93CF93DF93CDB7C7
:10472000DEB7AA970FB6F894DEBF0FBECDBFEAEB97
:10473000F2E08091F100819322E0E23CF207C9F7B8
:104740000E94F71E8091E80083FF2EC18091BA027B
:104750009091BB02492F50E04A30510508F024C126
:10476000FA01E558FF4F0C945225803821F0823829
:1047700009F01AC108C08091B6029091B70299233E
:1047800089F082600FC08091BE028F70873008F080
:104790000BC18093E9008091EB0085FB882780F9AD
:1047A0001092E9009091E800977F9093E800809341
:1047B000F1001092F100D1C0282F2D7F09F0F4C034
:1047C000882319F0823061F0EFC08091BC02813003
:1047D00009F0EAC0933009F080E08093B7022EC060
:1047E0008091BC0281112AC08091BE028F702FEF90
:1047F000280F263008F0D8C08093E9002091EB0004
:1048000020FF1CC0933021F48091EB00806214C023
:104810009091EB0090619093EB0021E030E0A901D2
:1048200002C0440F551F8A95E2F74093EA001092A8
:10483000EA008091EB0088608093EB001092E90021
:104840008091E800877F8093E8000E94A921ACC096
:104850008111AAC01091BC021F778091E30080787B
:10486000812B8093E3008091E800877F8093E800AC
:104870000E94A9218091E80080FFFCCF8091E30095
:1048800080688093E300111102C082E001C083E0E0
:104890008093B90289C08058823008F085C0809129
:1048A000BC029091BD028C3D53E0950779F583E001
:1048B0008A838AE289834FB7F894DE01139620E059
:1048C0003EE051E2E32FF0E050935700E49120FFE7
:1048D00003C0E295EF703F5FEF708E2F90E0EA30FB
:1048E00010F0C79601C0C0968D939D932F5F243121
:1048F00049F74FBF8091E800877F8093E8006AE224
:1049000070E0CE0101960E94B52016C06091BE02F3
:104910007091BF02AE014F5F5F4F0E94F91FBC0153
:10492000892B09F441C09091E800977F9093E800AB
:1049300089819A810E9413218091E8008B7780936E
:10494000E80032C0803881F58091E800877F80934D
:10495000E8008091B5028093F1008091E8008E77A5
:1049600072CF811121C08091BC029091BD02992724
:104970000297D4F48091E800877F8093E8008091CB
:10498000BC028093B5020E94A9218091B5028111D9
:1049900006C08091E30087FD02C081E001C084E091
:1049A0008093B9020E94E31E8091E80083FF0AC051
:1049B0008091E800877F8093E8008091EB0080621F
:1049C0008093EB00AA960FB6F894DEBF0FBECDBF62
:1049D000DF91CF911F9108950895CF938091B902EF
:1049E0008823A1F0C091E900CF709091EC00892F4D
:1049F000817090FD80E8C82B1092E9008091E8005A
:104A000083FD0E948C23CF70C093E900CF9108955D
:104A1000AA1BBB1B51E107C0AA1FBB1FA617B707E4
:104A200010F0A61BB70B881F991F5A95A9F7809500
:104A30009095BC01CD01089597FB072E16F40094C4
:104A400007D077FD09D00E94082507FC05D03EF469
:104A5000909581959F4F0895709561957F4F08952A
:104A6000A1E21A2EAA1BBB1BFD010DC0AA1FBB1F72
:104A7000EE1FFF1FA217B307E407F50720F0A21BE4
:104A8000B30BE40BF50B661F771F881F991F1A9451
:104A900069F760957095809590959B01AC01BD017B
:104AA000CF010895EE0FFF1F0590F491E02D0994BA
:104AB0008F929F92AF92BF92CF92DF92EF92FF922E
:104AC000CF93DF93EC01688179818A819B816115A5
:104AD00071058105910521F464E279ED8BE597E09C
:104AE0002DE133EF41E050E00E94132649015A01C5
:104AF0009B01AC01A7EAB1E40E9432266B017C0164
:104B0000ACEEB4EFA50194010E944026DC01CB017C
:104B10008C0D9D1DAE1DBF1DB7FF03C00197A109E0
:104B2000B04888839983AA83BB839F77DF91CF9115
:104B3000FF90EF90DF90CF90BF90AF909F908F90BD
:104B400008950E945825089580E091E00E9458251C
:104B50000895A0E0B0E08093000190930101A0933C
:104B60000201B09303010895FB01DC0104C08D91A3
:104B70000190801921F441505040C8F7881B990BCF
:104B80000895DC01CB01FC01F999FECF06C0F2BD0E
:104B9000E1BDF89A319600B40D9241505040B8F7FB
:104BA0000895F999FECF92BD81BDF89A992780B5F5
:104BB0000895A8E1B0E042E050E00C94C325DC0188
:104BC000A40FB51F4150504048F0CB01840F951FF2
:104BD0002E910E94F02541505040D0F70895262F85
:104BE000F999FECF92BD81BDF89A019700B40216E3
:104BF00039F01FBA20BD0FB6F894FA9AF99A0FBE91
:104C000008950396272F0E94F0250E94EF25252F57
:104C10000E94F025242F0C94F0250196272F0E9446
:104C2000F0250C94EF25052E97FB1EF400940E94AE
:104C30002A2657FD07D00E94302507FC03D04EF4EA
:104C40000C942A2650954095309521953F4F4F4F13
:104C50005F4F089590958095709561957F4F8F4F28
:104C60009F4F08950E944526A59F900DB49F900DDB
:104C7000A49F800D911D11240895B7FF0C94322636
:104C80000E943226821B930B0895A29FB001B39F0E
:104C9000C001A39F700D811D1124911DB29F700D45
:0C4CA000811D1124911D0895F894FFCF90
:104CAC0001000000FF0000FFFF0000FF7FFF00007D
:104CBC00FF0000FF0000FF0000FF000000000000EC
:104CCC000000000000FF2BFF55FF80FFABFFD5FF5E
:104CDC00C8002202451E491EBD1EB91EB51E481E27
:104CEC0001E200E900EA00B500B600B700CD008390
:104CFC0001CC008A01920194012102230224022595
:104D0C0002260227022A02B300B4006F0070008151
:104D1C008283E200E900EA00B500B600B700CD00DE
:104D2C008301CC008A019201940121022302240206
:104D3C002502260227022A02B300B4006F0070007D
:0A4D4C008182839435F49766F60027
:00000001FF
